:020000040800F2
:100000009009002065010008E90A00084D04000875
:1000100000000000000000000000000000000000E0
:10002000000000000000000000000000ED0A0008D1
:100030000000000000000000EB0A00080D0C0008A2
:1000400077010008770100087701000877010008B0
:1000500077010008770100087701000877010008A0
:1000600077010008770100087701000845040008BF
:100070007701000877010008770100087701000880
:100080007701000877010008770100087701000870
:100090007701000877010008770100087701000860
:1000A0007701000877010008770100087701000850
:1000B0007701000877010008770100087701000840
:1000C00000F002F800F03EF80CA030C80838241800
:1000D0002D18A246671EAB4654465D46AC4201D180
:1000E00000F030F87E460F3E0FCCB6460126334274
:1000F00000D0FB1AA246AB4633431847E00C000081
:10010000000D0000103A02D378C878C1FAD852071F
:1001100001D330C830C101D504680C6070470000BD
:100120000023002400250026103A01D378C1FBD813
:10013000520700D330C100D50B6070471FB51FBDFB
:1001400010B510BD00F041F91146FFF7F7FF00F0C0
:10015000BBFD00F059F903B4FFF7F2FF03BC00F058
:100160005DF900000748804707480047FEE7FEE7C3
:10017000FEE7FEE7FEE7FEE704480549054A064BB1
:1001800070470000810C0008C100000890030020A7
:1001900090090020900500209005002001E004C097
:1001A000091F0429FBD28B0701D50280801CC907D7
:1001B00000D00270704700290BD0C30702D0027034
:1001C000401C491E022904D3830702D50280801CEB
:1001D000891EE3E70022EEE70022DFE700220309A1
:1001E0008B4273D3030A8B4258D3030B8B423CD30D
:1001F000030C8B4221D312E003460B437FD4002231
:1002000043088B4274D303098B425FD3030A8B42AA
:1002100044D3030B8B4228D3030C8B420DD3FF2214
:10022000090212BA030C8B4202D31212090265D0E2
:10023000030B8B4219D300E0090AC30B8B4201D395
:10024000CB03C01A5241830B8B4201D38B03C01ADC
:100250005241430B8B4201D34B03C01A5241030B53
:100260008B4201D30B03C01A5241C30A8B4201D304
:10027000CB02C01A5241830A8B4201D38B02C01AAF
:100280005241430A8B4201D34B02C01A5241030A26
:100290008B4201D30B02C01A5241CDD2C3098B420B
:1002A00001D3CB01C01A524183098B4201D38B0188
:1002B000C01A524143098B4201D34B01C01A52412B
:1002C00003098B4201D30B01C01A5241C3088B4270
:1002D00001D3CB00C01A524183088B4201D38B005B
:1002E000C01A524143088B4201D34B00C01A5241FD
:1002F000411A00D201465241104670475DE0CA0FD4
:1003000000D04942031000D34042534000229C4693
:1003100003098B422DD3030A8B4212D3FC2289019D
:1003200012BA030A8B420CD3890192118B4208D373
:10033000890192118B4204D389013AD0921100E0D5
:100340008909C3098B4201D3CB01C01A52418309E9
:100350008B4201D38B01C01A524143098B4201D316
:100360004B01C01A524103098B4201D30B01C01A41
:100370005241C3088B4201D3CB00C01A52418308BB
:100380008B4201D38B00C01A5241D9D243088B4211
:1003900001D34B00C01A5241411A00D201466346B4
:1003A00052415B10104601D34042002B00D5494218
:1003B000704763465B1000D3404201B50020C04641
:1003C000C04602BD704770477047754600F022F87E
:1003D000AE46050069465346C008C000854618B0C1
:1003E00020B5FFF7C9FE60BC00274908B6460026C5
:1003F000C0C5C0C5C0C5C0C5C0C5C0C5C0C5C0C5D5
:10040000403D49008D4670470446C046C0462046E0
:10041000FFF7A1FE004870472C0300200149182077
:10042000ABBEFEE726000200704700000120034932
:100430000004486002490120486070470000024003
:100440000000002010B5FFF7F1FF10BDFEE700002F
:1004500010B5034A8021916200F0CAFB10BD000074
:100460000004004870B50D460646064980208861A4
:10047000002404E0305D00F0BBFB641CA4B2AC427D
:10048000F8D370BD0004004870B50C46054610490D
:10049000802088610F4E0F210902304600F0A4F938
:1004A000002230460DE05100695A83689B07DB0F3C
:1004B000FBD0C160C16881680906C90FFBD1521C1D
:1004C00092B2A242EFD30721090200F08DF970BD6C
:1004D000000400480038004010B51120FFF7B8FFB5
:1004E000962000F08FF92920FFF7B2FF962000F048
:1004F00089F910BDF8B51446104F4022069E1D46DE
:10050000BA624A19521E93B20219521E92B200F0F8
:100510005FF88020B86120000BD4094942008E5258
:10052000401EFBD505E02146054800F0E1FA6D1EAE
:10053000ADB2002DF7D14020B861F8BD00040048ED
:100540000C00002070B500F071F900F05BFA052195
:10055000134800F093F813480168402631430160C6
:1005600000F026F8FFF7B8FF104D0F4CAE62207870
:10057000641C411ECEB200280CD02078641CFFF70A
:1005800067FF31462046FFF76DFFA4190A2000F0EF
:1005900039F9ECE74020A861282000F035F870BD5B
:1005A00000000240003800406A0D000800040048C6
:1005B00010B5064C0820A0620A2000F023F908209C
:1005C000A061322000F01EF910BD000000040048B8
:1005D000F8B507461C4615460E462A20FFF738FF99
:1005E0006846078045800221FFF74EFF2B20FFF76A
:1005F0002FFF6846068044800221FFF745FF2C202C
:10060000FFF726FFF8BD000031B568460378FF21EB
:1006100041310C48F022282B10D0E82B0ED042801C
:100620000180094C4020A0623620FFF711FF012114
:100630006846FFF717FF4020A06138BD4180028067
:10064000EFE70000000000200004004808B504495E
:100650004A6902434A6149690140009108BD0000AE
:100660000010024008B50449CA690243CA61C96959
:100670000140009108BD000000100240044A5118DA
:100680002039C97F4258520852004250704700003A
:10069000630D0008F0B400230A68002A51D0012439
:1006A0000A689C402240002A47D04C68012C01D0A7
:1006B000022C10D18D681446866864436700E719E0
:1006C000BE436C4326438660CD680C684668A643EB
:1006D0006C43264346600F691446C6686443650050
:1006E0006519AC46AE4325467D432E43C6604D6832
:1006F000022D1BD1FF2A0CD84F691646056A2246E7
:10070000724372431601B61AB5437A431543056224
:100710000CE04E69150A2A466A436A436A4315018A
:10072000476AAD1AAF437243174347624A68056888
:100730006646B5435443254305605B1C0A68DA40AE
:10074000ADD1F0BC0020704710B57D21C900FFF786
:1007500045FD0449401E486100208861052008616C
:1007600010BD000000E000E030B4012203685B0629
:10077000DB0FD402002B2DD14B680A680D691A4398
:10078000CB682B431A434B691A438B691A43CB69D5
:100790001A430B6A1A430368114D2B401A43026037
:1007A0004268104B1A404B691B0C1A438B681A4362
:1007B00042608A68A24204D2630042689A431A43A4
:1007C000426001230A6A5B039A4202D1898C89B292
:1007D00001610022C169A143C16130BC104670476C
:1007E0004000FFFFFBF0FFFF42680F231B029A430C
:1007F0000A434260704700000149086070470000EA
:100800000800002081B008490A690092421C00D00B
:10081000401C002805D00A69D20300D5401E0028DC
:10082000F9D101B07047000000E000E008B50948C8
:10083000012142690A43426140690840009006482C
:1008400001680902090A016001200449C002086028
:1008500008BD00000010024008E400E000E100E0F4
:10086000F0B587B018216846FFF7B6FC0120C00438
:10087000FFF7ECFE01208005FFF7E8FE0120800471
:10088000FFF7E4FE01204004FFF7E0FE01201B4DCE
:100890008002A8620821A9622021A9624021A962E0
:1008A0008021A9620124032600276946D1C1694637
:1008B00028460494FFF7EEFE08206946D1C1694638
:1008C00028460494FFF7E6FE20206946D1C1694618
:1008D00028460494FFF7DEFE40206946D1C16946F0
:1008E00028460494FFF7D6FE80206946D1C16946A8
:1008F00028460494FFF7CEFE07B0F0BD0004004880
:10090000F0B591B0282106A8FFF766FC18216846CB
:10091000FFF762FC0127BF033846FFF7A3FE38014B
:10092000FFF794FE00247810022503260394049414
:100930006A46059461C269462D48FFF7ABFE0097F1
:100940000394049469462A48029601950594FFF79A
:10095000A1FEA803039404946A46059461C2694603
:100960002348FFF797FE244922480B791025C258E7
:10097000224E32402A43C2500A79835803252D0360
:10098000AB4383500B79C2582025AA43C2500B7940
:10099000C2584025AA43C2500D79425980239A4338
:1009A0001A4342510B798515C25803263602B243C9
:1009B0002A43C250097903154258B500AA431A4385
:1009C000425028010690FF200530079007200002C2
:1009D000089058100B900A94072009940F900C94DB
:1009E0000D940E9406A90648FFF7BEFE11B0F0BDA7
:1009F00000040048000002405C0D0008EFBFFFFF4C
:100A00000038004070B592B028216846FFF7E4FB3B
:100A100018210AA8FFF7E0FB2D480121C2698903CC
:100A20000A43C261C06900240840109007204003B7
:100A30000A9002200B9003200C900AA90D942548DF
:100A4000FFF728FE254924480D7910224359244EEA
:100A50003340134343510A79835803252D03AB4395
:100A600083500B79C2582025AA43C2500B79C25833
:100A70004025AA43C2500D79425980239A431A4314
:100A800042510B798515C25803263602B2432A43D8
:100A9000C2500A7903158158B500A9431943815002
:100AA00028010090FF2005300190072000020290ED
:100AB0005810059004940720039409900694079415
:100AC000089469460748FFF74FFE12B070BD00005A
:100AD000001002400004004800000240630D0008BE
:100AE000EFBFFFFF00380040FEE77047704700008F
:100AF000F3B50F46394C0F2181B009022046FFF7AC
:100B000073FE2168402081432160354D0521284630
:100B1000FFF7B4FD601568608000686060680226B9
:100B2000304360602F4C2079295831432950207977
:100B30002958082211432950052128461B3CFFF75C
:100B40009DFDE17F281D0A58120C12043A430A50F9
:100B5000E37F2248EA5801990C30234F3A40204F56
:100B60000C37102A34D03A1F9950E17FC851E07FEA
:100B70002958012211432950184F38684021084351
:100B800038601A4841680029FCD0002141600521E5
:100B90002846FFF773FD3A68384640218A433A6099
:100BA000CA006A604A016A607A68B2437A60E27F8A
:100BB000AB58B343AB50E27FAB580824A343AB50D0
:100BC00002680A43026007210902FFF70DFEFEBD1D
:100BD000D9510349E27F08315050C8E7003800403E
:100BE00000000240630D00081040000000000020DB
:100BF00005498A689207D20FFBD00873C8688868D5
:100C00000006C00FFBD1704700380040704700005D
:100C100010B5184801684908490001600168C90712
:100C2000C90FFBD11448016801221143016001681A
:100C30008907C90FFBD00168F82291438022114334
:100C400001604168F022914341604168072212022D
:100C50009143416041688908890041600C224168E4
:100C60001142FCD1054C2046FFF76EFD2046FFF7F0
:100C7000C3FD10BD002002400010024000127A00A7
:100C8000704700008307FF22DB0E9A408907090E98
:100C90009940002808DB830809489B001B18186846
:100CA00090430843186070470007000F0838830816
:100CB00004489B001B18D86990430843D8617047CB
:100CC00000E400E000ED00E008B52248012182695F
:100CD0000A4382618069084000900807FFF7C2FC60
:100CE0000321081FFFF7CEFFFFF792FFFFF7B8FDC4
:100CF0000120FFF7ABFC00210B20FFF7C3FF012011
:100D00001549C0020860FFF7FBFD6420FFF77AFD7C
:100D1000FFF718FC7D20C000FFF774FD0020FF22C4
:100D2000C823413201460090FFF7E4FB6420FFF73F
:100D300069FD552464021420FFF764FD1420FFF7B9
:100D400061FD64230A211A4608460094FFF7D2FB8E
:100D5000F1E700000010024000E100E0081C304410
:100D6000586C80081C3044586C8004EF03800204E7
:100D7000CF00C13005ED6403128104E885007806D8
:100D8000CB392C00340202F72003EA000002C02312
:100D900002C11003C53E2802C7860236480237004A
:100DA000023A5503B1001804B608822702F2000285
:100DB000260110E00F312B0C0E084EF137071003FF
:100DC0000E090010E1000E1403110731C148080F8D
:100DD0000C31360F0211800229800000FC0D000842
:100DE000000000200C00000004010008080E0008AC
:100DF0000C00002084090000200100084001F000E0
:080E00000000000000127A005E
:04000005080000C12E
:00000001FF
